:0400000002074B3276
:03000B0002067A70
:0100130032BA
:01001B0032B2
:0100230032AA
:01002B0032A2
:10074B0075810F120747E582600302003302003305
:1000330012069780FEAA82AB83C295C2977C00C347
:10004300EC64809490501F8A058B067D00530680D4
:10005300ED4EC36001B39296D297C297EBCA25E0E7
:10006300CA33FB0C80D9D295C29522900A0512009F
:1000730038900B07120038900900120038900C01D9
:10008300120038900F001200382212006E85576953
:10009300756A00AA697401456AFB8A828B83120020
:1000A30038855869756A00AA697402456AFB8A82B1
:1000B3008B83120038855969756A00AA69740345F0
:1000C3006AFB8A828B83120038855A69756A00AA93
:1000D300697404456AFB8A828B83120038855B69E5
:1000E300756A00AA697405456AFB8A828B831200CC
:1000F30038855C69756A00AA697406456AFB8A8259
:100103008B83120038855D69756A00AA6974074597
:100113006AFB8A828B83120038855E69756A00AA3E
:10012300697408456AFB8A828B8312003822E54E84
:1001330030E103120564E54E30E30312057EE54E1C
:1001430030E403120598E54E30E5031205B822E5C5
:1001530058B47E03755800E55AB47E03755A00E51A
:100163005CB47E03755C00E55EB47E03755E0022BD
:10017300E535B4FF030201F0E535640AC0E0740A13
:1001830030E702F404F5F0E53530E702F40484F5D2
:10019300F0D0E020D20930E706C3E495F0F5F0AAE9
:1001A300F0EA90071193FA8A5EE535640AC0E074B9
:1001B3000A30E702F404F5F0E53530E702F404848D
:1001C300D0E020D20930E706C3E495F0F5F0AAF0B9
:1001D300EA90071193FA8A5DE54F30E3087480458E
:1001E3005DF55D800E747F555DF55D8006755D017F
:1001F300755E01E534B4FF03020273E534640AC09B
:10020300E0740A30E702F404F5F0E53430E702F471
:100213000484F5F0D0E020D20930E706C3E495F07A
:10022300F5F0AAF0EA90071193FA8A5CE534640AC0
:10023300C0E0740A30E702F404F5F0E53430E70275
:10024300F40484D0E020D20930E706C3E495F0F546
:10025300F0AAF0EA90071193FA8A5BE54F30E208BF
:100263007480455BF55B800E747F555BF55B8006A0
:10027300755B01755C01E533B4FF030202F6E533F8
:10028300640AC0E0740A30E702F404F5F0E53330A1
:10029300E702F40484F5F0D0E020D20930E706C386
:1002A300E495F0F5F0AAF0EA90071193FA8A5AE57B
:1002B30033640AC0E0740A30E702F404F5F0E5336E
:1002C30030E702F40484D0E020D20930E706C3E427
:1002D30095F0F5F0AAF0EA90071193FA8A59E54FE1
:1002E30030E10874804559F559800E747F5559F5EE
:1002F300598006755A01755901E532B4FF030203AB
:1003030079E532640AC0E0740A30E702F404F5F0D8
:10031300E53230E702F40484F5F0D0E020D209306E
:10032300E706C3E495F0F5F0AAF0EA90071193FA13
:100333008A58E532640AC0E0740A30E702F404F52F
:10034300F0E53230E702F40484D0E020D20930E74C
:1003530006C3E495F0F5F0AAF0EA90071193FA8A40
:1003630057E54F30E00874804557F557800E747F8A
:100373005557F557800675580175570112015222DA
:1003830012017312013112008D22E53355325534B7
:100393005535FABAFF140544C3E544940A400B905B
:1003A3000C00120038C2AF75870222E532B4FF0297
:1003B3008038E5326027754400755300434E02D2FE
:1003C30094053CE4B53C02053DC3E53C943CE53D66
:1003D3009400401FE4F53DF53C15328016C2947538
:1003E3005301534EFD534FFE8009534EFD534FFEB1
:1003F30075530022E533B4FF028038E53360277577
:100403004400755400434E08D293053EE4B53E02C2
:10041300053FC3E53E943CE53F9400401FE4F53FB0
:10042300F53E15338016C293755401534EF7534F5F
:10043300FD8009534EF7534FFD75540022E534B444
:10044300FF028032E5346024754400434E10D2929B
:100453000540E4B540020541C3E5409410E54194ED
:100463000E4019E4F541F54015348010C292534E05
:10047300EF534FFB8006534EEF534FFB22E535B44A
:10048300FF028032E5356024754400434E20C2915B
:100493000542E4B542020543C3E542943CE5439477
:1004A30000401BE4F543F54215358012D291534EBB
:1004B300DF534FF78008534EDF534FF7D291220596
:1004C30049C3E549946440127549001203AE12030F
:1004D300F712044012048012038D227401554EFA60
:1004E300BA0002800302055720B218434E01C3E548
:1004F3004A940A4003754A00AA4A054AEA90071B30
:1005030093F53220B318434E01C3E54B940A4003DD
:10051300754B00AA4B054BEA90072593F53320B49E
:1005230018434E01C3E54C940E4003754C00AA4C8E
:10053300054CEA90072F93F53420B518434E01C3B9
:10054300E54D940A4003754D00AA4D054DEA900709
:100553003D93F53522743C55B0FABA3C03534EFE35
:10056300220545C3E54594144003534FFEC3E545B7
:1005730094644006434F01754500220546C3E54692
:1005830094144003534FFDC3E54694644006434F20
:1005930002754600220547C3E54794144003534FB1
:1005A300FBAA477B00C3EA94C8EB94004006434F81
:1005B30004754700220548C3E54894144003534F8C
:1005C300F7C3E54894644006434F0875480022AAE0
:1005D30082EA6004C2B08002D2B022AA82EA600436
:1005E300C2B18002D2B122AA821536E536600280FA
:1005F3000F05390539E539B502037539007537003B
:1006030022AA82153AE53A6002800F053B053BE5D5
:100613003BB50203753B0075380022E5536027E5BF
:100623003760028019E53990070993FA8A82120527
:10063300D27401253990070993F536753701758210
:10064300041205EA8002D2B022E5546027E538603F
:10065300028019E53B90070D93FA8A821205DE7436
:1006630001253B90070D93F53A7538017582041205
:1006730006048002D2B122C0E0C0F0C082C083C0B1
:10068300D075D008438CDC0530D0D0D083D082D055
:10069300F0D0E032754F00754E0075B0FF7590FFD6
:1006A300758901D28CD2A9D2AF7535FF7534FF7528
:1006B30033FF7532FFE4F543F542E4F541F540E4D9
:1006C300F53FF53EE4F53DF53C753B0075390075A6
:1006D3004D00754C00754B00754A00753800753731
:1006E30000755400755300754400E53060FC7530A7
:1006F300001204DE1204C212055812038312061EEE
:1007030012064C80E52201140064011400147E30AB
:100713006D79335B5F707F7BFF0003050A0F14194C
:100723001E00FF0003050A0F14191E00FF0001023B
:10073300030508090A0B0C0D0E00FF0003050A0F41
:0807430014191E00758200224A
:00000001FF
